:0200000480007A
:100000006F008004732F2034930F80006308FF0378
:10001000930F90006304FF03930FB0006300FF038E
:10002000130F000063040F0067000F00732F2034CC
:1000300063540F006F00400093E19153171F0000BD
:1000400023223FFC6FF09FFF732540F163100500F2
:10005000970200009382020173905230735000188F
:10006000970200009382020273905230B702008020
:100070009382F2FF7390023B9302F0017390023A75
:1000800097020000938282017390523073502030A7
:1000900073503030735040309301000097020000DD
:1000A000938282F673905230130510001315F501F8
:1000B000634C05000F00F00F930110009308D0056A
:1000C000130500007300000093020000638E02001D
:1000D00073905210B7B20000938292107390223046
:1000E00073232030E39A62F47350003097020000CB
:1000F0009382420173901234732540F173002030D3
:10010000B70000801301000033D72040B70E0080F5
:10011000930120006314D759B70000801301100029
:1001200033D72040B70E00C0930130006318D75773
:10013000B70000801301700033D72040B70E00FFD6
:1001400093014000631CD755B70000801301E00005
:1001500033D72040B70EFEFF930150006310D755F0
:10016000B7000080938010001301F00133D72040C6
:10017000930EF0FF930160006312D753B700008025
:100180009380F0FF1301000033D72040B70E0080AA
:10019000938EFEFF930170006312D751B700008069
:1001A0009380F0FF1301100033D72040B70E0040BA
:1001B000938EFEFF930180006312D74FB70000803B
:1001C0009380F0FF1301700033D72040B70E000179
:1001D000938EFEFF930190006312D74DB70000800D
:1001E0009380F0FF1301E00033D72040B70E0200E8
:1001F000938EFEFF9301A0006312D74BB7000080DF
:100200009380F0FF1301F00133D72040930E0000DC
:100210009301B0006314D749B7808181938010188F
:100220001301000033D72040B78E8181938E1E18B2
:100230009301C0006314D747B78081819380101861
:100240001301100033D72040B7CEC0C0938E0E0CE0
:100250009301D0006314D745B78081819380101833
:100260001301700033D72040B70E03FF938E3E304A
:100270009301E0006314D743B78081819380101805
:100280001301E00033D72040B70EFEFF938E6E605F
:100290009301F0006314D741B780818193801018D7
:1002A0001301F00133D72040930EF0FF93010001BA
:1002B0006316D73FB780818193801018130100FC2B
:1002C00033D72040B78E8181938E1E189301100181
:1002D0006316D73DB780818193801018130110FCFD
:1002E00033D72040B7CEC0C0938E0E0C93012001AF
:1002F0006316D73BB780818193801018130170FC7F
:1003000033D72040B70E03FF938E3E309301300168
:100310006316D739B7808181938010181301E0FCF0
:1003200033D72040B70EFEFF938E6E6093014001DD
:100330006316D737B7808181938010181301F0FFBF
:1003400033D72040930EF0FF930150016318D73547
:10035000B700008013017000B3D02040B70E00FF3B
:1003600093016001639CD033B70000801301E0006B
:1003700033D12040B70EFEFF930170016310D133DB
:1003800093007000B3D01040930E000093018001E1
:100390006396D03113020000B70000801301700093
:1003A00033D72040130307001302120093022000EA
:1003B000E31452FEB70E00FF930190016310D32F98
:1003C00013020000B70000801301E00033D7204083
:1003D0001300000013030700130212009302200011
:1003E000E31252FEB70EFEFF9301A0016318D32B58
:1003F00013020000B70000801301F00133D7204042
:100400001300000013000000130307001302120082
:1004100093022000E31052FE930EF0FF9301B0010F
:10042000631ED32713020000B70000801301700081
:1004300033D720401302120093022000E31652FE2D
:10044000B70E00FF9301C001631AD7251302000005
:10045000B70000801301E0001300000033D72040F4
:100460001302120093022000E31452FEB70EFEFFA7
:100470009301D0016314D72313020000B70000805A
:100480001301F001130000001300000033D72040D7
:100490001302120093022000E31252FE930EF0FFAB
:1004A0009301E001631CD71F13020000B700008016
:1004B000130000001301700033D720401302120014
:1004C00093022000E31452FEB70E00FF9301F001E7
:1004D0006316D71D13020000B70000801300000050
:1004E0001301E0001300000033D720401302120074
:1004F00093022000E31252FEB70EFEFF93010002AA
:10050000631ED71913020000B7000080130000001B
:10051000130000001301F00133D720401302120032
:1005200093022000E31252FE930EF0FF930110029B
:100530006316D7171302000013017000B700008084
:1005400033D720401302120093022000E31652FE1C
:10055000B70E00FF930120026312D71513020000AB
:100560001301E000B70000801300000033D72040E3
:100570001302120093022000E31452FEB70EFEFF96
:1005800093013002631CD711130200001301F00124
:10059000B7000080130000001300000033D7204094
:1005A0001302120093022000E31252FE930EF0FF9A
:1005B000930140026314D70F13020000130170006F
:1005C00013000000B700008033D720401302120050
:1005D00093022000E31452FEB70E00FF9301500275
:1005E000631ED70B130200001301E000130000008C
:1005F000B70000801300000033D720401302120020
:1006000093022000E31252FEB70EFEFF9301600238
:100610006316D709130200001301F0011300000054
:1006200013000000B700008033D7204013021200EF
:1006300093022000E31252FE930EF0FF930170022A
:10064000631ED7059300F00033511040930E000055
:10065000930180026314D1059300000233D100405E
:10066000930E000293019002631AD103B35000402D
:10067000930E00009301A0026392D0039300004008
:10068000371100001301018033D02040930E000089
:100690009301B0026314D001631030020F00F00F19
:1006A000638001009391110093E111009308D0053C
:1006B00013850100730000000F00F00F930110007C
:1006C0009308D0051305000073000000731000C0EC
:1006D000000000000000000000000000000000001A
:1006E000000000000000000000000000000000000A
:0C06F000000000000000000000000000FE
:1010000000000000000000000000000000000000E0
:1010100000000000000000000000000000000000D0
:1010200000000000000000000000000000000000C0
:1010300000000000000000000000000000000000B0
:081040000000000000000000A8
:040000058000000077
:00000001FF
